:020000040000FA
:060000000219FD02031CC1
:03000B0002008D63
:03001300020535AE
:03001B0002009050
:03002B000202D1FD
:03005B0002054457
:030073000203097C
:100080000406080C10182030406080A0C0054032E3
:10009000C2AFC2A853E6EFC28E856B8BC0D0D2D35D
:1000A000C0E0C0F0C2CAA8CCA9CDD2CAD2AF758A6E
:1000B00000C3E8956CF8E9956DF9C3E913F9E81305
:1000C000F8E5666007C3E913F9E813F8E97025E875
:1000D000956E4020956E501CE582B410177C007B15
:1000E000007A007908900000A86AE5667004C3E809
:1000F00013F801FD900000D2A8D2AA61E7E0FDC389
:100100009CC39840EF98EB33FB0582E0FCC39DC392
:100110009840E198EB33FB0582E0FDC39CC3984017
:10012000D398EB33FB0582E0FCC39DC39840C59890
:10013000EB33FB0582E0FDC39CC39840B798EB33DB
:10014000FB0582E0FCC39DC39840A998EB33FB05F7
:1001500082E0FDC39CC398409B98EB33FB0582E093
:10016000FCC39DC398408D98EB33FB0582217890AA
:100170000000D2A8D2AA61E7E0FDC39CC39840EF7B
:1001800098EA33FA0582E0FCC39DC39840E198EAFF
:1001900033FA0582E0FDC39CC39840D398EA33FA52
:1001A0000582E0FCC39DC39840C598EA33FA0582F6
:1001B000E0FDC39CC39840B798EA33FA0582E0FC9F
:1001C000C39DC39840A998EA33FA0582E0FDC39C19
:1001D000C398409B98EA33FA0582E0FCC39DC3981C
:1001E000408D98EA33FA0582EBC46B6A54F0F9EA61
:1001F000C454F0C3996009900000D2A8D2AA61E764
:10020000EBF4C454F0F9EAF4C4540F49FAEBF4C423
:10021000540FFBC3EAF99460FAEB9400FB5020C33F
:10022000E97B007A0079006016C3135006F9C39584
:1002300052600AE9F5527553007900800205533087
:100240003A27C3EA94D0F8EB9407F9400BE8FAE9AF
:10025000FB203509D235415D303502C235203902E7
:10026000B235C3EA33FAEB33FBEB2B3B3BF9C3EB81
:1002700013FBEA13FAEA29FAEB3400FB30E3047AC1
:10028000FF7BFFE5255403601B202A18E55D33F949
:10029000EB7007C3E99A4002E9FAE53CC4332AFA55
:1002A000EB3400FBC3EA33C4540FF8EB33C454F00F
:1002B00048F87005EA60027801900000D2A8D2AA3E
:1002C000E5226002152281D4900000D2A8D2AA6152
:1002D000E7C0D0C0E0C2CF0541E5666009E56560D2
:1002E000057565006104756501E52360021523C38A
:1002F000E55460057555006104E5552401F5555038
:10030000037555FFD0E0D0D032C2AF53E67F75926F
:10031000FA7593FFC22053917FD2AF32C0E0E58AD5
:10032000303408856B8BF0A3D0E032D0E0C2AF53FD
:10033000E6EFC0D0C0E0C0F0D2D3D2AF5388EFA870
:100340008AA98CAA40308D010A758A00758C0075C7
:100350004000438810E566700AC3E833F8E933F9D2
:10036000EA33FA30331FE8C4540FFAE9C454F04AB0
:10037000FAC3132AFAC3E833F8E933F9E82AFAE9A9
:100380003406FB61D830320FC3E833E933FAE82A88
:10039000FAE93400FB61D8303115E875F056A4AAAB
:1003A000F0E975F056A42AFAC5F03400FB61D8C311
:1003B000EA13FAE913F9E813F8E875F056A4AAF07D
:1003C000E975F056A42AFAC5F03400C313FBEA130A
:1003D000FAC3EB13FBEA13FAC3EB94125009C3EA16
:1003E0009434EB940750160522E52270021522C3BF
:1003F000E52294325002A128755400A12BE5226019
:100400000215223036067C007D088117AC31AD32F2
:10041000303A04AC33AD34C3EA9CFAEB9DFB92084E
:10042000AE60AF61303A425007203509D235813590
:10043000303502C235303504AE62AF63203902B2C6
:1004400035C3EA33FAEB33FBA208500AEAF424017D
:10045000FAEBF43400FBC3EA9450FAEB9400FB503F
:100460001478007A007B008175A208500878007A21
:10047000007B0081D4E5255403601B202A18E55D2C
:1004800033F9EB7007C3E99A4002E9FAE53CC4335B
:100490002AFAEB3400FBEA8EF0A4F9AAF0EB8EF016
:1004A000A42AFAC5F03400FBC3EB13FDEA13F8C32A
:1004B000ED13FDE813F80FEF146004C3E833F8C33D
:1004C000E933EA33FAEB33FBDFEDEB30E30678FF99
:1004D0007AFF7B078854D230E86003755500C3E586
:1004E0005BFC955C4002AC5CC3EC95545008EC7529
:1004F000F008A4FAABF0EAF4F8EBF45407F9C3E817
:10050000948CFAE99400FB50047A007B00885689A9
:10051000578A588B5975230AD0F0D0E0D0D053F7C2
:10052000DF43F74043E6103275230AD0F0D0E0D025
:10053000D043E61032C2AAD28EC2CA85CC6C85CD19
:100540006DD2CA32C2AFC0D0C0E0D2D3A8F9E55A4A
:1005500030E20AE5FA20E23520E132A165E5FA3021
:10056000E22B20E128C3E55713F8E55613F5FB8885
:10057000FCC3E55913F8E55813F5E988EA85575A9D
:1005800053F7BFD2A8303402D2AA53E6EF53F7DFB5
:10059000D0E0D0D0D2AF32790180147903801079C5
:1005A0000A800C791E80087964800479C8800078FC
:1005B00017E4D5E0FDD8FAD9F62278FF202828796B
:1005C000A1E76023E548601F74FF8548F084853FFC
:1005D000F030290375F005A4F8C5F0600278FFC378
:1005E000E8955D5002A85D885C22C3E54794A0E5CC
:1005F000489400E55C500314A1FB046002F55C2202
:1006000075E89022055EC3E55E9408405330EDF432
:10061000A8BDA9BE755E00E9FA79A0E76041EA705D
:1006200006E55F6018800CC3E8955F600EE55F50DB
:1006300005600A1480070460FA8002E55FF55FC375
:100640009569401B755BC0C394044013755B80C300
:100650009404400B755B40C394044003755B002217
:10066000E55B2410500274FFF55B22743279A68793
:10067000F0A4C5F0A2F733F55D227547007548F088
:1006800022C2AFC2CAA8CCA9CDAA4130CF010AD29A
:10069000CAD2AFC3EA13FAE913F9E813F8AB42ACD4
:1006A0004388428943C3E89BF8E99C20280A547F89
:1006B000F9302C02E19FC1F8AD448A44F9EA9D5417
:1006C0007FFA600678FF79FFC1DDAE45AF468B4506
:1006D0008C46A842A943C3E89EF8E99FF9C3E548C0
:1006E00013FBE54713FAE82AF547E93BF5485006BE
:1006F0007547FF7548FFE145AA47AB48AC47AD4891
:100700007E047F02C3EB9404400D1E1FC3EB9408CC
:1007100040052029021E1FC3ED13FDEC13FCDEF77C
:10072000C3EA9CFAEB9DFBEF6009C3E913F9E813F8
:10073000F8DFF7EA28FAEB39FB8A478B4850067B4B
:10074000FF8B478B48C3EB94025002D22C30280415
:100750007F03E1707892E6FFC3E53D948240110F7C
:10076000C3E53D94A040010FC3EF940640027F050E
:100770007E02E548C4540FF9E548C454F0F8E54753
:10078000C4540F28F8C3E89EFAE99400FB4009C35B
:10079000EA9401EB940050047A01E4FB0207EBAA0F
:1007A00047AB48EBC4FEEAC4540F4EFCC3EA9CFAC4
:1007B000EB9400FBC3E813C313F8EA28FAEB340008
:1007C000FB8A478B48C3EB94024002C22C7802EBB1
:1007D000C4FE7B00EAC4540F4EFAC3EA98FA4005FF
:1007E000C3940150027A017892E6FF302002E1EBD7
:1007F000854E92854F93D22043E680C3E49AF8E475
:100800009BF9C3E833F8E933F9302C03020880E898
:10081000FAE9FBD3E913FDE813FC884E894FC3EFD7
:1008200094036038EF20E00CE82CF8E93DF9ECFA8D
:10083000EDFB8013E828F8E939F9C3E82401F8E969
:100840003400F97AFF7BFFC3EF9403400F8A508B8B
:1008500051884A894B8C4C8D4D0208B5885089517E
:100860008A4A8B4B8C4C8D4D3028127550F0755147
:10087000FF754CF0754DFF754EF0754FFF0208B5D2
:10088000E8FAD3E813FC884EC3EF94036021EF200D
:10089000E007E82CF8ECFA01A0E8282401F87AFF38
:1008A000C3EF940340098A50884A8C4C0208B588EB
:1008B000508A4A8C4C30200201B5753A02D220434E
:1008C000E680E5255403602DA847A948C3E913F93C
:1008D000E813F8302804E92440F9C2AF53E67F75E5
:1008E0009100C3E498F594E499F595759104D220AC
:1008F00043E680D2AF22D221754900752000302B0B
:10090000037520402114D221754900752040302BF9
:100910000375200078017901202C20E5255403601F
:1009200002C2217914E548C313700104F8C394147A
:1009300040027814302804781B791BC3E833F8C3CD
:10094000E933F9202010E549600C302803D53A043A
:10095000D22221C711BD0549E5BF5440B52002216F
:10096000B130280908C3E899400118214320210A21
:1009700008C3E899400221142143C22153E67F7540
:100980009100302C117594007595F0759104D2206A
:1009900043E680020914E5487EFFC3334009C333B0
:1009A0004005C3334001FEC3E49E759400F59521D4
:1009B0008BC3E5399401500221143021022114D84F
:1009C0000221C52143C222C2AF53E67F7591008543
:1009D0005094855195759104854A92854B93D22008
:1009E00043E680D2AFE5255403600720290205398C
:1009F000801030220D202B0A20210715811581023D
:100A000014052278003021027801E53D75F007A435
:100A1000F9E5F028F5F0E9A2F013A2F113A2F21320
:100A2000F53DC394785003753D78C3E53D953E4050
:100A30000CC285C286C28775D4FF75D507302002E7
:100A4000413D854C92854D93D22043E6802220384B
:100A500013C2AFC291D29075D47F75D503D2AF7552
:100A6000AA536142C2AFC291D29275D4DF75D50646
:100A7000D2AF75AA536142203813C2AFC28775D472
:100A8000BF75D505D290D2AF75AA436142C2AFC23D
:100A90008575D4BF75D505D292D2AF75AA63614270
:100AA000203813C2AFC290D29275D4BF75D505D28B
:100AB000AF75AA636142C2AFC292D29075D4BF75BE
:100AC000D505D2AF75AA438079203813C2AFC2864C
:100AD00075D4DF75D506D292D2AF75AA538063C2A2
:100AE000AFC28675D47F75D503D290D2AF75AA53A5
:100AF0008050203813C2AFC292D29175D4DF75D521
:100B000006D2AF75AA43803AC2AFC290D29175D4D3
:100B10007F75D503D2AF75AA638027203813C2AF83
:100B2000C28575D47F75D503D291D2AF75AA638083
:100B300011C2AFC28775D4DF75D506D291D2AF7519
:100B4000AA43227A147B7880127A107B8C800C7AEC
:100B50000D7BB480067A0B7BC88000E564D5E0018C
:100B6000227902E4C291D5E0FDD286D5E0FDC286AD
:100B7000D5E0FDD291D5E0FDE920E002D28530E05C
:100B800002D287E564D5E0FDE920E002C28530E0CD
:100B900002C2877496D5E0FDD9C9EAF8D5E0FDD840
:100BA000FBDBB8C29122C285C286C287C290C291C5
:100BB000C29275D4FF75D50722788076FF0876FF3C
:100BC0000876FF0876FF0876FF0876FF08760908A2
:100BD00076FF087601788C76010876FF0876FF08A4
:100BE00076FF0876FF0876FF0876030876FF08761A
:100BF000FF0876FF0876250876D008762808765014
:100C00000876040876FF0876020876FF08767A08E8
:100C100076FF0876070876010876FF0876FF0876E3
:100C20000008760022FA75F00CA4ABF0EAC333F8A2
:100C3000740133F9E8C333F8E933F9E8C32BF8E971
:100C40003400F9E8C333F8E933F9227888E6C3942D
:100C500003D23A5002C23AC238E630E102D238A298
:100C60003892397886E6149000809378A6F67886D4
:100C7000E6F53FC394025003753F02789CE6753E4B
:100C8000FFB40203753EA0B40303753E8278A0E66C
:100C9000F8600674282409D8FCF5697896E6912551
:100CA00088318932789EE69125883389347897E6B1
:100CB00091258835893671A6223036117A007B005D
:100CC0007CFF7D007E00B11F8B618A6022303A225A
:100CD0007896E6FA7B00789EE6FC7D00C3EA33FA5C
:100CE000EB33FBC3EC33FCED33FD7E0AB11F8B63AA
:100CF0008A627896303A02789EE6FA7B007897E628
:100D0000FC7D007E00303A10C3EA33FAEB33FBC3BC
:100D1000EC33FCED33FD7E0AB11F8B618A6022C388
:100D2000EC9EFCED9400FDC3EC9AFCED9BFDC3EC46
:100D30009423ED940050047C237D00C3EC94FFEDDC
:100D4000940140047CFF7D017BFF0B7A000AEA706E
:100D500009C3EC33FCED33FDA14AEC8AF0A4AEF0FC
:100D6000ED8AF0A42E947C40E4EAF460DD22D236D1
:100D700091B91205A31205A37A007B007C1012051D
:100D80009BE5542AFA74003BFBDCF37C04C3EB13B1
:100D9000FBEA13FADCF7FFEB60027FFFC23691B982
:100DA0002278A5E6F95403D2837002C283E9540C79
:100DB000D2847002C284E954307000E954C07000DB
:100DC000227567007568007597DE7597AD7581C0EF
:100DD00043FF8075EF0675A90071A675800275F155
:100DE000FF75A4F875800275D4FF75900075F20741
:100DF00075A50775900075D50775A60175E3407553
:100E0000E20271A6E4F8F6D8FD71B9121449789897
:100E10008664753001C2AF1205AB71431205A37130
:100E2000491205A3714F1205A3B1A1C2AF756700A6
:100E300075680078FA79FA308107D9FBD8F7021C77
:100E400000914B91B97898866471A675A91375A71E
:100E50001075C10075A70075660075E401758811ED
:100E6000758E0475890975C80475910475D8407527
:100E7000D90875F782759E0375960275DA4275DB9F
:100E80004275A82375E69075B80175BF8075AB00F3
:100E900075D10C75BCB975BB1075E88075B20112BF
:100EA0000597D2AF753C00C2301205ABC231C232D9
:100EB000C233C2347552007553007522001205A763
:100EC000C3E522940A5002E191D231752200120545
:100ED000A7C3E522940A5002E191C231D2327522B1
:100EE000001205A7C3E522940A5002E19175E4912E
:100EF000758851758E017589AA758C00758D00C233
:100F0000A9D2ABD2AA756B80756A14756E50C232C5
:100F1000D23475220A1205A7756A10C3E522940A15
:100F20007552007553004069758E0C756B00756ABB
:100F300028756E2875220A1205A7756A20C3E52256
:100F4000940A7552007553004047758E0C756B807E
:100F5000756A14756E1475220A1205A7756A10C396
:100F6000E522940A755200755300402575E4017519
:100F70008811758E04758909D2A9C2ABC2AAC23480
:100F8000D2337522001205A7C3E522940A4002C19C
:100F90002B12059B203003020E2BC2AF714371430D
:100FA0007143D2AF1205AB203403303A030210551F
:100FB00012059B788CE6C394015003021055E5306E
:100FC000C3940150030210557567A57568F17F023F
:100FD000D23691B91205A7C2AFC23691B9C3E55452
:100FE000947FD2AF406F120597C2AF7155D2AFDF79
:100FF000DFB16EC3EF7897F61205AB1215367F0A94
:10100000D236120CB91205A7C2AFC236120CB9C340
:10101000E554947FD2AF50E6120597C2AF120B434E
:1010200012059F120B43D2AFDFD6120D6EEF2403D1
:101030007896F6F87997E7C394234003985006E82A
:1010400024237897F61205AB9190B1651205A7128B
:101050000CB9020E2B7567007568001205A7C3E571
:101060005494014003020FA7C2AF120B55120B5547
:10107000120B55D2AF1205AB753000E4F537F538D9
:101080000537E537F4703F0538789AE6781914602B
:1010900012783214600D787D14600878FA146003B9
:1010A000753800C3E53898401D120BA61205971538
:1010B0003875370078998664C2AF120B55D2AF7875
:1010C0009886641205A712059FE5237003020E2B74
:1010D000C3E5549401500AC3E5529401501602101E
:1010E000801205A7E5237003020E2B75520075537D
:1010F00000021296C3E55294017017C2AF120BA6FC
:1011000078998664120B4378988664D2AF1205A74B
:101110004188C3E55294027017C2AF120BA67899AA
:101120008664120B4978988664D2AF1205A741886D
:10113000C3E55294037017C2AF120BA67899866468
:10114000120B4F78988664D2AF1205A74188C3E589
:101150005294047017C2AF120BA678998664120BD2
:101160005578988664D2AF1205A74188C3E552949A
:10117000057017C2AF120BA678998664120B5578CA
:10118000988664D2AF1205A74188C3E552940770D0
:1011900019C3E5539406500201D07401303A027429
:1011A000037888F6C238C2394188C3E55294087082
:1011B00019C3E5539406500201D07402303A027408
:1011C000047888F6D238D2394188C3E55294097040
:1011D00017C3E5539406500201D0303A0BC3788808
:1011E000E69402F6C23A4188C3E552940A7016C3E7
:1011F000E5539406500201D0203A0A7888E624028A
:10120000F6D23A4188C3E55294147025C3E553944D
:1012100006500201D0C2AF901A0B740093D2AF787F
:1012200088F613C238C2394002D2384002D239801F
:1012300057C3E55294157038C3E5539406404FC226
:10124000AF901A0B740093D2AFF8B801027402B8D1
:1012500002027401B803027404B8040274037888AB
:10126000F613C238C2394002D2384002D23980184F
:10127000C3E552940C70117567A57568F1C3E55309
:101280009406400A9190D2AF75520075530075676D
:101290000075680001D0C2AF120BA6E4D2AFE4F52E
:1012A0005EF524F525F53D755E08120597120600DA
:1012B00030EDFDA8BDA9BEE97001F8885F120604F3
:1012C000755E08C2AF12066B855D5B855D5CD2AF53
:1012D00075A71075C13075A70075A9037566013033
:1012E0003A07C238303502D238D228753900120A8E
:1012F000F2120B1B12067A12068112067A1206816E
:1013000012067A120906120A03120A4E12068112F6
:1013100008F6202C031205BA302C031205EA120A33
:1013200003120A77120681120906120A03120AA092
:101330001206811208F6120A03120AC91206811255
:101340000906120A03120AF2120681120600120896
:10135000F6120A03120B1B1206041206813028270C
:10136000855D5B79187A0CC3E53999400EC228D2A5
:10137000298A3B855D5B855D5C800CC3E5549401E7
:101380004003021303810D30291F202B1CE53B1461
:101390007006C229D22A6103F53B203A07C3E554FF
:1013A000940140030213038064753C00203A0F78D7
:1013B000FA79A4E760027803C3E55598504FE52316
:1013C000604B303A17203805203507800F30350242
:1013D000800A202B07D22B855D5B613378F0302BA0
:1013E00005855D5B7820C3E5489850030213033000
:1013F0002B1BC22BC238303502D238D229753B1292
:10140000855D5B6103053CE55460028110753C001D
:10141000C2AF120BA675240075250075A91375A718
:101420001075C10075A700756600D2AF1205A7122E
:101430000BA678A4E66006D290D291D292C3E53C86
:1014400094044003020E2B017B901A0D782091C961
:10145000E520B4550AA391C9E520B4AA028013750A
:1014600067A57568F1120BB99190756700756800F2
:10147000801D901A0378807B0A91C9A308DBFA903B
:101480001A0F788C7B1A91C9A308DBFA901A2922CB
:10149000C2AFB10C91E9901A00741091CEA37407F9
:1014A00091CEA3742191CE901A0378807B0A91CDBE
:1014B000A308DBFA901A0F788C7B1A91CDA308DB76
:1014C000FAB11F91FD901A2922E493F622E6438F88
:1014D00001538FFDFFC3E583941C400122EF856714
:1014E000B78568B7F0538FFE22438F02438F018583
:1014F00067B78568B7901A0DF0538FFC22901A0DCC
:10150000745591CE901A0E74AA91CE227A3079D069
:101510007820901A4091C9E520F709A3DAF7227ADA
:101520003079D0901A40E791CE09A3DAF9227C05F0
:101530001205ABDCFB22C2AF120B43120B49120B9C
:101540004F120B5512059F120B43120B49120B4FF2
:10155000120B5512059F120B43120B49120B4F121F
:101560000B55D2AF22C2AF120B55120B4F120B49C3
:10157000120B4312059F120B55120B4F120B4912FF
:101580000B4312059F120B55120B4F120B49120BF6
:0415900043D2AF2271
:1019FD00020DC1100721FFFFFFFFFFFF09FF01FFD0
:101A0D0055AA01FFFFFFFFFF03FFFFFF25D0285061
:0D1A1D0004FF02FF7AFF0701FFFF0000FF3A
:101A400023515F485F373023202020202020202092
:101A500023424C48454C492445464D3842323123B7
:101A60002020202020202020202020202020202076
:101C0000C2AFC2D37597DE7597AD7581C075A90057
:101C100043FF80752438752503B1DB7529A5752A26
:101C2000F143F10253A4FDD28175D4FF75E3407DE9
:101C3000FA780379E67C10752200752300901DE880
:101C40007B06752498752501308102814820810822
:101C5000D8FBD9F9DCF781BA308108D8FBD9F9DC97
:101C6000F781BAB19BE493A3C39A6004DDC381BA40
:101C7000DBDBB18D600281317B08E493FAA3B16EA6
:101C8000DBF87A30B16E752200752300B18DEAFC65
:101C9000EBFDC3ED94FE400EB18D8A278B28ED300D
:101CA000E0048A828B83B18D7AC270D8C3ED94FE32
:101CB000601950CEBD0029EC600F7520007521FF22
:101CC000752900752A000200008100A827A92808AC
:101CD00009D804D90281DDB191EAF281D10D81A642
:101CE000C3ED94035051EDA2E092007AC5C3E582A2
:101CF0009400E583941C508C200010438F02438F86
:101D0000018529B7852AB7F0300027A827A9280818
:101D100009438F01538FFDD804D902A132C3E58353
:101D2000941C4003A3A117E28529B7852AB7F0A325
:101D3000A117538FFC81827AC1BD030CE493A3FAEF
:101D4000B152DCF8B14A81828184AA22AB23B16E00
:101D5000EBFAEA6222752608C3E52313F523E52290
:101D600013F52250066323A0632201D526EAB1DBD6
:101D7000B1DB75260AEAF4200102D281300102C2E9
:101D800081B1DBC3134002C201D526EB22B191EA37
:101D9000FB208102A191308102A196752608AE2414
:101DA000AF25C3EF13FFEE13FEB1DFB1DBC3EA13C0
:101DB0003081024480FA30E703632201C3E5231334
:101DC000F523E52213F52250066323A0632201D5F3
:101DD00026D9E52265236523F52222AE24AF250E00
:101DE0000FDEFEDFFCD20122424C48656C693437BD
:061DF0003164E8B20601B7
:00000001FF
